:020000040000FA
:06000000C5EF16F012002E
:06080000C5EF16F0120026
:06082A000100F02D0000AA
:0808300000010000D9000000E6
:08083800D9CFE6FFE1CFD9FFA3
:10084000040EE126DE6ADE6ADE6ADD6ADD52DD5212
:10085000FD0EDBCF14F0FE0EDBCF15F0166A176A23
:1008600015AE02D016681768D9CFE9FFDACFEAFFD4
:10087000030EEB501718E8AE02D0173408D014500E
:10088000EE5C1550EE581650EE581750EE580FE229
:100890000C0EE66EA5EC16F0E552D9CFE9FFDACFE3
:1008A000EAFFEE2A000EEE22EE22EE22D1D7040E4F
:1008B000E15C02E2E16AE552E16EE552E7CFD9FF81
:1008C00012000F0EC16E070EB46E936A816A300E6D
:1008D000926E80900F0E946EF19E1200D9CFE6FFBB
:1008E000E1CFD9FF020EE1268250020B01E0010E9A
:1008F000080DF3CF16F08250010B040DF3CF15F065
:100900008050200B01E0010EE824146E8050100B83
:1009100001E0010E142415241624DE6EDD6ADECFFC
:1009200014F0DDCF15F014C0F3FF15C0F4FF020E74
:10093000E15C03E200D0E16AE552E16EE552E7CF07
:10094000D9FF12008092320EE66EE1EC16F0E5520D
:100950008084320EE66EE1EC16F0E5528094320EA1
:10096000E66EE1EC16F0E55212008082010EE66EB2
:10097000E66A62DFE552E5528084010EE66EE66AC1
:100980005BDFE552E5528094010EE66EE66A54DFC5
:10099000E552E5521200380E816ED4DF320EE66E5B
:1009A000E66A4ADFE552E552010E816ECBDF320E78
:1009B000E66EE66A41DFE552E5520D0E816EC2DF5A
:1009C000320EE66EE66A38DFE552E552060E816EBB
:1009D000B9DF320EE66EE66A2FDFE552E55212000D
:1009E000010E816EAFDF0A0EE66EE66A25DFE55284
:1009F000E5521200D9CFE6FFE1CFD9FF020E816E9A
:100A0000A1DF0A0EE66EE66A17DFE552E552FD0E3B
:100A1000DBCFE6FFFE0EDB50280DF350E552E72456
:100A2000E76EFE0EE7CFDBFFFD0EDB6AFE0EDB504E
:100A3000F36EFD0EDBCFF4FFF350F45C0BE2140E0B
:100A4000816E80DF320EE66EE1EC16F0E552FD0EAF
:100A5000DB2AECD7E552E7CFD9FF1200D9CFE6FF6A
:100A6000E1CFD9FFFE0EDB50816E7FDF010EE66E17
:100A7000E66AE2DEE552E552E552E7CFD9FF120021
:100A8000D9CFE6FFE1CFD9FFFD0EDBCFE9FFFE0EA8
:100A9000DBCFEAFFEF500EE0FD0EDBCFE9FFDB2AF4
:100AA000FE0EDBCFEAFF01E3DB2AEF50E66ED6DF76
:100AB000E552EAD7E552E7CFD9FF12000101DD6B1D
:100AC000300E926EF00E936EEF0ED96FD9C181FF8A
:100AD000040EDA6FDA51000821E2D951FE0BE84228
:100AE000D96FD9C181FF050EE66EE66AA5DEE55233
:100AF000E5528150100B09E08150200B06E0815037
:100B0000400B03E08150800B01E10AD80101DD05B3
:100B100002E1DE5104D0DA05DA6FDCD7CFD712005C
:100B2000F00E936E81CFDCF10101DC15DB6F0F0E4F
:100B3000D915D96FD951DB11D96F81CFDCF1F00E06
:100B4000DC15DB6FF00EDB5D01E0F7D7936A06D8AA
:100B5000DFC1DEF10101010EDD6F12000101E06B6A
:100B6000100EE05D14E2E051EA6A000FE96E010E3A
:100B7000EA22EF50D95D08E1E051EA6A100FE96E10
:100B8000010EEA22EFCFDFF1E029E06FE9D7DFC104
:100B900081FF640EE66EE66A4FDEE552E552120012
:100BA0000101E16B070EE15D1DE288DF0101E26FEB
:100BB000E151EA6AE30FE96E010EEA22E2C1EFFFBA
:100BC000E151EA6AE30FE96E010EEA22EF504608AE
:100BD00002E108D004D0E2C1E6FF40DFE5520101A6
:100BE000E12BE0D7E151EA6AE30FE96E010EEA2258
:100BF000EF6A12000101E16B070EE15D16E2E151BF
:100C0000EA6AE30FE96E010EEA22EF50E66E26DF94
:100C1000E5520101E129EA6AE30FE96E010EEA22D9
:100C2000EF5001E102D0E12BE7D71200D9CFE6FF68
:100C3000E1CFD9FFE652F250800B01E0010EDF6EEA
:100C4000F29EA69EA69CA684FE0EDB50A96EFD0E0B
:100C5000DB50A86E550EA76EAA0EA76EA682A6B28E
:100C6000FED7A694DF50E8B0F28EE8A0F29EE552DF
:100C7000E552E7CFD9FF1200D9CFE6FFE1CFD9FF88
:100C8000A69CA69EFE0EDB50A96EA680A85000D0A2
:100C9000E552E7CFD9FF1200D9CFE6FFE1CFD9FF68
:100CA000020EE126DE6ADD6ADECF14F0DDCF15F03C
:100CB000D890155004E6050E145C000E155824E279
:100CC000FD0EDBCF14F0FE0EDBCF15F0DE5014244A
:100CD000E96EDD501520EA6EEF50E66EDE50010140
:100CE00020250F01E96EDD50010121210F01EA6E7F
:100CF000800EE926000EEA22E552E750EF6EDF2A69
:100D0000010E01E3DB2AD0D7050E01012025206F5B
:100D1000000E2121216F020EE15C02E2E16AE55240
:100D2000E16EE552E7CFD9FF1200D9CFE6FFE1CF60
:100D3000D9FF070EE126FE0EDB50390A02E126EF4D
:100D40000DF0010A02E1FAEF0CF00F0A02E1CEEF1A
:100D50000CF0010A02E1A2EF0CF0030A02E176EFC7
:100D60000CF0010A02E14AEF0CF0070A02E11EEF63
:100D70000CF0010A02E1F2EF0BF0030A02E1C6EF08
:100D80000BF0010A02E19AEF0BF06A0A02E16EEF42
:100D90000BF0030A02E142EF0BF0010A02E116EF49
:100DA0000BF00F0A02E1EAEF0AF0010A01E1E6D3D3
:100DB000030A01E1B7D3010A01E188D3070A01E17F
:100DC00059D3010A01E12AD3030A01E1FBD2010A46
:100DD00001E1CCD21F0A01E19DD2010A01E16ED2EC
:100DE000030A01E13FD2010A01E10FD2070A01E142
:100DF000DFD1010A01E1AFD1030A01E17FD1010A8C
:100E000001E14FD10F0A01E11FD1010A01E1EFD049
:100E1000030A01E1BFD0010A01E18FD0070A60E0B7
:100E2000010A31E0030A02E052EF0DF0DE6ADD6AEA
:100E3000DECF14F0DDCF15F0D890155004E6050E86
:100E4000145C000E15581DE2DECFE9FFDDCFEAFF8E
:100E5000250EE926010EEA22EF50E66ED950020F68
:100E6000146EDACF15F0DE501424E96EDD50152033
:100E7000EA6EE552E750EF6EDF2A010E01E3DB2A4E
:100E8000D7D752EF0DF0DE6ADD6ADECF14F0DDCF8A
:100E900015F0D890155004E6050E145C000E155898
:100EA0001DE2DECFE9FFDDCFEAFF2A0EE926010EC3
:100EB000EA22EF50E66ED950020F146EDACF15F029
:100EC000DE501424E96EDD501520EA6EE552E7503D
:100ED000EF6EDF2A010E01E3DB2AD7D752EF0DF0C8
:100EE000DE6ADD6ADECF14F0DDCF15F0D890155044
:100EF00004E6050E145C000E15581DE2DECFE9FF76
:100F0000DDCFEAFF2F0EE926010EEA22EF50E66E52
:100F1000D950020F146EDACF15F0DE501424E96EAA
:100F2000DD501520EA6EE552E750EF6EDF2A010E24
:100F300001E3DB2AD7D752EF0DF0DE6ADD6ADECFA0
:100F400014F0DDCF15F0D890155004E6050E145CB2
:100F5000000E15581DE2DECFE9FFDDCFEAFF340EAB
:100F6000E926010EEA22EF50E66ED950020F146E08
:100F7000DACF15F0DE501424E96EDD501520EA6E4C
:100F8000E552E750EF6EDF2A010E01E3DB2AD7D7E7
:100F900052EF0DF0DE6ADD6ADECF14F0DDCF15F022
:100FA000D890155004E6050E145C000E15581DE28D
:100FB000DECFE9FFDDCFEAFF390EE926010EEA2296
:100FC000EF50E66ED950020F146EDACF15F0DE50F6
:100FD0001424E96EDD501520EA6EE552E750EF6EFD
:100FE000DF2A010E01E3DB2AD7D752EF0DF0DE6ACC
:100FF000DD6ADECF14F0DDCF15F0D890155004E691
:10100000050E145C000E15581DE2DECFE9FFDDCFA2
:10101000EAFF3E0EE926010EEA22EF50E66ED950B5
:10102000020F146EDACF15F0DE501424E96EDD5095
:101030001520EA6EE552E750EF6EDF2A010E01E35C
:10104000DB2AD7D752EF0DF0DE6ADD6ADECF14F06F
:10105000DDCF15F0D890155004E6050E145C000E97
:1010600015581DE2DECFE9FFDDCFEAFF430EE9268A
:10107000010EEA22EF50E66ED950020F146EDACF5D
:1010800015F0DE501424E96EDD501520EA6EE552AD
:10109000E750EF6EDF2A010E01E3DB2AD7D752EFCC
:1010A0000DF0DE6ADD6ADECF14F0DDCF15F0D890EA
:1010B000155004E6050E145C000E15581DE2DECF37
:1010C000E9FFDDCFEAFF480EE926010EEA22EF50E4
:1010D000E66ED950020F146EDACF15F0DE501424EC
:1010E000E96EDD501520EA6EE552E750EF6EDF2A1B
:1010F000010E01E3DB2AD7D752EF0DF0DE6ADD6A7D
:10110000DECF14F0DDCF15F0D890155004E6050EB3
:10111000145C000E15581DE2DECFE9FFDDCFEAFFBB
:101120004D0EE926010EEA22EF50E66ED950020F6D
:10113000146EDACF15F0DE501424E96EDD50152060
:10114000EA6EE552E750EF6EDF2A010E01E3DB2A7B
:10115000D7D752EF0DF0DE6ADD6ADECF14F0DDCFB7
:1011600015F0D890155004E6050E145C000E1558C5
:101170001DE2DECFE9FFDDCFEAFF520EE926010EC8
:10118000EA22EF50E66ED950020F146EDACF15F056
:10119000DE501424E96EDD501520EA6EE552E7506A
:1011A000EF6EDF2A010E01E3DB2AD7D752EF0DF0F5
:1011B000DE6ADD6ADECF14F0DDCF15F0D890155071
:1011C00004E6050E145C000E15581DE2DECFE9FFA3
:1011D000DDCFEAFF570EE926010EEA22EF50E66E58
:1011E000D950020F146EDACF15F0DE501424E96ED8
:1011F000DD501520EA6EE552E750EF6EDF2A010E52
:1012000001E3DB2AD7D752EF0DF0DE6ADD6ADECFCD
:1012100014F0DDCF15F0D890155004E6050E145CDF
:10122000000E15581DE2DECFE9FFDDCFEAFF5C0EB0
:10123000E926010EEA22EF50E66ED950020F146E35
:10124000DACF15F0DE501424E96EDD501520EA6E79
:10125000E552E750EF6EDF2A010E01E3DB2AD7D714
:1012600052EF0DF0DE6ADD6ADECF14F0DDCF15F04F
:10127000D890155004E6050E145C000E15581DE2BA
:10128000DECFE9FFDDCFEAFF610EE926010EEA229B
:10129000EF50E66ED950020F146EDACF15F0DE5023
:1012A0001424E96EDD501520EA6EE552E750EF6E2A
:1012B000DF2A010E01E3DB2AD7D7F4D3DE6ADD6A29
:1012C000DECF14F0DDCF15F0D890155004E6050EF2
:1012D000145C000E15581DE2DECFE9FFDDCFEAFFFA
:1012E000660EE926010EEA22EF50E66ED950020F93
:1012F000146EDACF15F0DE501424E96EDD5015209F
:10130000EA6EE552E750EF6EDF2A010E01E3DB2AB9
:10131000D7D7C8D3DE6ADD6ADECF14F0DDCF15F093
:10132000D890155004E6050E145C000E15581DE209
:10133000DECFE9FFDDCFEAFF6B0EE926010EEA22E0
:10134000EF50E66ED950020F146EDACF15F0DE5072
:101350001424E96EDD501520EA6EE552E750EF6E79
:10136000DF2A010E01E3DB2AD7D79CD3DE6ADD6AD0
:10137000DECF14F0DDCF15F0D890155004E6050E41
:10138000145C000E15581DE2DECFE9FFDDCFEAFF49
:10139000700EE926010EEA22EF50E66ED950020FD8
:1013A000146EDACF15F0DE501424E96EDD501520EE
:1013B000EA6EE552E750EF6EDF2A010E01E3DB2A09
:1013C000D7D770D3DE6ADD6ADECF14F0DDCF15F03B
:1013D000D890155004E6050E145C000E15581DE259
:1013E000DECFE9FFDDCFEAFF750EE926010EEA2226
:1013F000EF50E66ED950020F146EDACF15F0DE50C2
:101400001424E96EDD501520EA6EE552E750EF6EC8
:10141000DF2A010E01E3DB2AD7D744D3DE6ADD6A77
:10142000DECF14F0DDCF15F0D890155004E6050E90
:10143000145C000E15581DE2DECFE9FFDDCFEAFF98
:101440007A0EE926010EEA22EF50E66ED950020F1D
:10145000146EDACF15F0DE501424E96EDD5015203D
:10146000EA6EE552E750EF6EDF2A010E01E3DB2A58
:10147000D7D718D3DE6ADD6ADECF14F0DDCF15F0E2
:10148000D890155004E6050E145C000E15581DE2A8
:10149000DECFE9FFDDCFEAFF7F0EE926010EEA226B
:1014A000EF50E66ED950020F146EDACF15F0DE5011
:1014B0001424E96EDD501520EA6EE552E750EF6E18
:1014C000DF2A010E01E3DB2AD7D7ECD2DE6ADD6A20
:1014D000DECF14F0DDCF15F0D890155004E6050EE0
:1014E000145C000E15581DE2DECFE9FFDDCFEAFFE8
:1014F000840EE926010EEA22EF50E66ED950020F63
:10150000146EDACF15F0DE501424E96EDD5015208C
:10151000EA6EE552E750EF6EDF2A010E01E3DB2AA7
:10152000D7D7C0D2DE6ADD6ADECF14F0DDCF15F08A
:10153000D890155004E6050E145C000E15581DE2F7
:10154000DECFE9FFDDCFEAFF890EE926010EEA22B0
:10155000EF50E66ED950020F146EDACF15F0DE5060
:101560001424E96EDD501520EA6EE552E750EF6E67
:10157000DF2A010E01E3DB2AD7D794D2DE6ADD6AC7
:10158000DECF14F0DDCF15F0D890155004E6050E2F
:10159000145C000E15581DE2DECFE9FFDDCFEAFF37
:1015A0008E0EE926010EEA22EF50E66ED950020FA8
:1015B000146EDACF15F0DE501424E96EDD501520DC
:1015C000EA6EE552E750EF6EDF2A010E01E3DB2AF7
:1015D000D7D768D2DE6ADD6ADECF14F0DDCF15F032
:1015E000D890155004E6050E145C000E15581DE247
:1015F000DECFE9FFDDCFEAFF930EE926010EEA22F6
:10160000EF50E66ED950020F146EDACF15F0DE50AF
:101610001424E96EDD501520EA6EE552E750EF6EB6
:10162000DF2A010E01E3DB2AD7D73CD2DE6ADD6A6E
:10163000DECF14F0DDCF15F0D890155004E6050E7E
:10164000145C000E15581DE2DECFE9FFDDCFEAFF86
:10165000980EE926010EEA22EF50E66ED950020FED
:10166000146EDACF15F0DE501424E96EDD5015202B
:10167000EA6EE552E750EF6EDF2A010E01E3DB2A46
:10168000D7D710D2DE6ADD6ADECF14F0DDCF15F0D9
:10169000D890155004E6050E145C000E15581DE296
:1016A000DECFE9FFDDCFEAFF9D0EE926010EEA223B
:1016B000EF50E66ED950020F146EDACF15F0DE50FF
:1016C0001424E96EDD501520EA6EE552E750EF6E06
:1016D000DF2A010E01E3DB2AD7D7E4D1DE6ADD6A17
:1016E000DECF14F0DDCF15F0D890155004E6050ECE
:1016F000145C000E15581DE2DECFE9FFDDCFEAFFD6
:10170000A20EE926010EEA22EF50E66ED950020F32
:10171000146EDACF15F0DE501424E96EDD5015207A
:10172000EA6EE552E750EF6EDF2A010E01E3DB2A95
:10173000D7D7B8D1DE6ADD6ADECF14F0DDCF15F081
:10174000D890155004E6050E145C000E15581DE2E5
:10175000DECFE9FFDDCFEAFFA70EE926010EEA2280
:10176000EF50E66ED950020F146EDACF15F0DE504E
:101770001424E96EDD501520EA6EE552E750EF6E55
:10178000DF2A010E01E3DB2AD7D78CD1DE6ADD6ABE
:10179000DECF14F0DDCF15F0D890155004E6050E1D
:1017A000145C000E15581DE2DECFE9FFDDCFEAFF25
:1017B000AC0EE926010EEA22EF50E66ED950020F78
:1017C000146EDACF15F0DE501424E96EDD501520CA
:1017D000EA6EE552E750EF6EDF2A010E01E3DB2AE5
:1017E000D7D760D1DE6ADD6ADECF14F0DDCF15F029
:1017F000D890155004E6050E145C000E15581DE235
:10180000DECFE9FFDDCFEAFFB10EE926010EEA22C5
:10181000EF50E66ED950020F146EDACF15F0DE509D
:101820001424E96EDD501520EA6EE552E750EF6EA4
:10183000DF2A010E01E3DB2AD7D734D1DE6ADD6A65
:10184000DECF14F0DDCF15F0D890155004E6050E6C
:10185000145C000E15581DE2DECFE9FFDDCFEAFF74
:10186000B60EE926010EEA22EF50E66ED950020FBD
:10187000146EDACF15F0DE501424E96EDD50152019
:10188000EA6EE552E750EF6EDF2A010E01E3DB2A34
:10189000D7D708D1DE6ADD6ADECF14F0DDCF15F0D0
:1018A000D890155004E6050E145C000E15581DE284
:1018B000DECFE9FFDDCFEAFFBB0EE926010EEA220B
:1018C000EF50E66ED950020F146EDACF15F0DE50ED
:1018D0001424E96EDD501520EA6EE552E750EF6EF4
:1018E000DF2A010E01E3DB2AD7D7DCD0DE6ADD6A0E
:1018F000DECF14F0DDCF15F0D890155004E6050EBC
:10190000145C000E15581DE2DECFE9FFDDCFEAFFC3
:10191000C00EE926010EEA22EF50E66ED950020F02
:10192000146EDACF15F0DE501424E96EDD50152068
:10193000EA6EE552E750EF6EDF2A010E01E3DB2A83
:10194000D7D7B0D0DE6ADD6ADECF14F0DDCF15F078
:10195000D890155004E6050E145C000E15581DE2D3
:10196000DECFE9FFDDCFEAFFC50EE926010EEA2250
:10197000EF50E66ED950020F146EDACF15F0DE503C
:101980001424E96EDD501520EA6EE552E750EF6E43
:10199000DF2A010E01E3DB2AD7D784D0DE6ADD6AB5
:1019A000DECF14F0DDCF15F0D890155004E6050E0B
:1019B000145C000E15581DE2DECFE9FFDDCFEAFF13
:1019C000CA0EE926010EEA22EF50E66ED950020F48
:1019D000146EDACF15F0DE501424E96EDD501520B8
:1019E000EA6EE552E750EF6EDF2A010E01E3DB2AD3
:1019F000D7D758D0DE6ADD6ADECF14F0DDCF15F020
:101A0000D890155004E6050E145C000E15581DE222
:101A1000DECFE9FFDDCFEAFFCF0EE926010EEA2295
:101A2000EF50E66ED950020F146EDACF15F0DE508B
:101A30001424E96EDD501520EA6EE552E750EF6E92
:101A4000DF2A010E01E3DB2AD7D72CD0DE6ADD6A5C
:101A5000DECF14F0DDCF15F0D890155004E6050E5A
:101A6000145C000E15581DE2DECFE9FFDDCFEAFF62
:101A7000D40EE926010EEA22EF50E66ED950020F8D
:101A8000146EDACF15F0DE501424E96EDD50152007
:101A9000EA6EE552E750EF6EDF2A010E01E3DB2A22
:101AA000D7D700D0D950020FE66E000EDA20E66ECE
:101AB0004CEC06F0E552E552070EE15C02E2E16A09
:101AC000E552E16EE552E7CFD9FF120061EC04F078
:101AD000FF0E0101F215F26FF36BF2C1F4F1F3C1E5
:101AE000F5F1060E0D6E0E6AF4C108F0F5C109F0AD
:101AF0000AEC15F008C0F4F109C0F5F1816A220E74
:101B0000E66E010EE66E3FEC14F0E552E552F3CFBF
:101B1000F8F1F4CFF9F10101F451F81902E1F551AE
:101B2000F91901E135D0010EF825F86F000EF92101
:101B3000F96F0A0EF9AF02D0D89003D0F85D000E0D
:101B4000F95903E20101232B23D0640EF81901E1B6
:101B5000F95105E10101300E226F236F19D0F8C150
:101B6000E6FFF9C1E6FFE90E146E2D0E156E166A3A
:101B700014C0E6FF15C0E6FF16C0E6FF220EE66EB3
:101B8000010EE66EB4EC14F0176E070EE15E17500E
:101B90000101206B216B0101EE6BEF6B020EEFAFC9
:101BA00002D0D89003D0EE5D000EEF5910E2220E65
:101BB000EE25E96E010EEF21EA6EEF50E66E95EC30
:101BC00006F0E5520101EE2B000EEF23E7D7F66B8E
:101BD000F76B040EF7AF02D0D89003D0F65D000E7D
:101BE000F7593AE2EC6BED6B806A80828092EC6B85
:101BF000ED6B0A0EEDAF02D0D89003D0EC5D000E75
:101C0000ED5926E2800EEC25E96E000EED21EA6E1C
:101C1000EF50816EF06BF16BC80EF1AF02D0D8902F
:101C200003D0F05D000EF15906E2F22B000EF32313
:101C3000F02BF123F1D7640EE66EE1EC16F0E552DD
:101C400080848094816A0101EC2B000EED23D1D7B2
:0C1C5000F62B000EF723BDD751D7120071
:041C5C006AEC13F02B
:101C6000FB0EDBCFF3FFDB06F35000090AE0B8EC14
:101C700013F0FA0E23EC14F0F3E1151CF1E1010E60
:101C800001D0000E99EF13F06AEC13F03B0EE12443
:101C900002E3E168E652E16E010EDB6A020EDB6AE6
:101CA000F90EDBCFF6FFFA0EDBCFF7FFFB0EDBCF33
:101CB000F8FF0800F550DF6EDF5002E1BDEF12F0D3
:101CC000250EDF5C02E0B0EF12F0030EDB6A040EBB
:101CD000DB6A050EDB6A060EDB6A070EDB6AD2ECF6
:101CE00012F02D0EDF5C0CE02B0EDF5C09E0200E05
:101CF000DF5C06E0230EDF5C03E0300EDF5C1AE100
:101D0000DF50300A14E0130A0FE0030A0AE00B0A5E
:101D100005E0060AE4E1030EDB80E1D7030EDB8277
:101D2000DED7030EDB84DBD7030EDB86D8D7030EAA
:101D3000DB88D5D72A0EDF5C1BE1CEEC12F01CEC61
:101D400013F010E0030EDB8008680968130EDBCF88
:101D50000DF0140EDBCF0EF030EC15F0040E06C0C3
:101D6000DBFF03D0130E05EC13F0D2EC12F00BD016
:101D7000090EDB6A73EC13F003E0E7EC13F0FAD71B
:101D8000090E05EC13F0030EDBB0DB982E0EDF5CC2
:101D90001BE1D2EC12F02A0EDF5C0BE1CEEC12F06C
:101DA0001CEC13F003E1130E57EC13F0D2EC12F01D
:101DB0000BD0090EDB6A73EC13F003E0E7EC13F0D1
:101DC000FAD7090E57EC13F0680EDF5C07E1D2EC8E
:101DD00012F0680EDF5C1DE1030E18D0740EDF5C9C
:101DE00017E07A0EDF5C14E0480EDF5C06E0540E6C
:101DF000DF5C03E05A0EDF5C02E1020E07D06C0EDE
:101E0000DF5C03E06A0EDF5C04E1010EAAEC13F074
:101E1000C9DBDF506E0A01E17FD31E0A01E192D1D6
:101E2000200A01E18FD13F0A01E149D11A0A01E1FB
:101E300046D10D0A01E143D1200A01E140D13A0A1D
:101E400001E13DD1200A01E13AD1260A01E135D173
:101E50000D0A01E132D11A0A01E1D9D0200A4AE083
:101E6000300A1FE0460A0EE0250A01E083D3D9506C
:101E7000F90FE96EFF0EDA20EA6E010EEE5E000E3B
:101E8000EE5AEE5AB8EC13F0250EE66E95DB03E140
:101E9000151C01E169D3B4EC13F001E26BD3DB2A2A
:101EA00069D3080EDB6A040EDB50010806E2040E5B
:101EB000DB047CEC13F0DB508BDB080EDB5009E01D
:101EC000030EDB50010B05E172DB01E04DD3080E80
:101ED000DB6A64DBEFCFDFFF2CEC14F003E1151CB1
:101EE00001E142D3B4EC13F001E3DB2A60DB01E152
:101EF00041D33AD3070EDB5002080FE1F8EC13F0A0
:101F0000030EBFEC13F00E0EEECFDBFF0F0EEECF85
:101F1000DBFF100EEECFDBFF20D0F70EDBCF17F08C
:101F2000F80EDBCF18F0020E175E000E185AF70EEF
:101F300017C0DBFFF80E18C0DBFF17C0E9FF18C0A1
:101F4000EAFFAFEC13F0166A0E0E14C0DBFF0F0EA3
:101F500015C0DBFF100E16C0DBFF0E0EDBCFE6FF59
:101F60000F0EDBCFE6FF100EDBCFE6FF34EC16F0F2
:101F7000E552E552E552130E07C0DBFF140E08C010
:101F8000DBFF060EDB5005E0130EF3EC13F001E26D
:101F90006ADB17EC14F002E2130E37DBDAEC13F015
:101FA00006E0040EF3EC13F002E2050E2EDB030E46
:101FB000DBB005D0FCDA01E0D7D2080EDB6A090EEF
:101FC000DB6A0E0EDBCFF6FF0F0EDBCFF7FF100E36
:101FD000DBCFF8FF0800F550DF6EDF5014E01DEC9A
:101FE00014F011E22CEC14F003E1151C01E1BCD259
:101FF000BBDB01E3DB2A090EDB2AD9500E0FE96EA9
:10200000000ECBDBE7D7D3DA01E1B4D2ADD2C6DA2A
:10201000110EEECFDBFF120EEDCFDBFF110EDBCF8B
:10202000E6FF120EDBCFE6FF26EC16F0E552E55296
:10203000130EF3CFDBFF140EF4CFDBFF060EDB50E5
:1020400004E0130ED0DB01E20EDB17EC14F002E229
:10205000130EDBDAAFDB05E0040EC5DB02E2050E92
:10206000D4DA030EDBB005D0A2DA01E07DD2080E8F
:10207000DB6A090EDB6A110EDBCFE9FF120EDBCF44
:10208000EAFFEFCFDFFFDF5014E0D7DB12E2E4DB43
:1020900003E1151C01E168D267DB01E3DB2A090ECD
:1020A000DB2A110EDB2ADBCFE9FF120EE8E3DB2A85
:1020B000E6D77DDA01E15ED257D2030EDB8E070E42
:1020C000DB0410E195DB040E5ADB0A0EEECFDBFFDA
:1020D0000B0EEECFDBFF0C0EEECFDBFF0D0EEECFC7
:1020E000DBFF6CD0070EDB5003082CE1030EDBAEE8
:1020F0000DD0B2DA020E76DAEFCF14F0156A166A56
:10210000176A14AE39D01568166835D0F70EDBCFD4
:1021100015F0F80EDBCF16F0020E155E000E165A03
:10212000F70E15C0DBFFF80E16C0DBFF15C0E9FF88
:1021300016C0EAFFEFCF14F00A0E14C0DBFF0B0E3F
:10214000DB6A38D0070EDB50020809E1030EDBAE74
:1021500004D059DB16AE10D00ED055DB0DD0030ED7
:10216000DBAE12D079DA020E3DDAF9DA166A176AB6
:1021700015AE02D016681768E2DA0C0E16C0DBFF47
:102180000D0E17C0DBFF1AD0F70EDBCF16F0F80EDE
:10219000DBCF17F0020E165E000E175AF70E16C0B0
:1021A000DBFFF80E17C0DBFF16C0E9FF17C0EAFF20
:1021B000D6DAC5DA0C0EDB6A0D0EDB6A060EDB50D2
:1021C00005E1010EF36E050EF3CFDBFF150EDB6AA2
:1021D000160EDB6AD950370F146E000EDA20156E1A
:1021E000390E14C0DBFF3A0E15C0DBFF380EDB6A78
:1021F000080EDB6A0A0EAEDADF50780A12E0200A17
:1022000010E0280A0CE0200A0AE03F0A06E00D0A66
:1022100002E0200A08E1020E05D0080E03D0080EE5
:10222000DF26100E97DA030EDBBE02D0DB92DB94C2
:10223000DB50800B24E08ADAD890030EEB50000AC2
:1022400008E6000EEE5C000EEE58000EEE58000E92
:10225000EE5815E213DA0B680C680D680E68EEECA8
:1022600015F00A0E02C0DBFF0B0E03C0DBFF0C0EE5
:1022700004C0DBFF0D0E05C0DBFF2D0E08D0030EE2
:10228000DBA202D02B0E03D0DBA408D0200EF36E0D
:10229000170EF3CFDBFF150EDB2A02D0170EDB6A19
:1022A000050EDB5003E1B7D901E189D0D80E146ED9
:1022B0002D0E156E000E166E070EDBCF17F0186A86
:1022C000196A1A6A17C00BF018C00CF019C00DF08B
:1022D0001AC00EF0D3D959EC16F014500224F36E44
:1022E00015500320F46E16500420F86EF4CFF7FF5B
:1022F000F3CFF6FF0800090EF5CFDBFF580EDF5CC9
:102300000FE1610EF36E090E7BD90AE3200E146E05
:10231000090EDBCFE7FF1450E75E090EE7CFDBFFC6
:10232000070EDBCF14F0156A166A176A0FDA14C0AD
:102330000BF015C00CF016C00DF017C00EF0EECF6C
:1023400006F0EECF07F0EECF08F0EFCF09F059EC32
:1023500016F009C0EDFF08C0EDFF07C0EDFF06C095
:10236000EFFF390EDBCFE9FFDB063A0EDBCFEAFFEA
:1023700001E2DB06090EDBCFEFFF150EDB2A4BD99E
:1023800095E1030EDBA61DD06F0EDF5C06E1C1D91F
:1023900018E3150EDB285BDA14D0780EDF5C09E059
:1023A000580EDF5C06E0620EDF5C03E0420EDF5C8D
:1023B00008E1020EF36E160EF3CFDBFF02D0150E0E
:1023C000DB6A030EDB50100B0EE0040EDBCF14F0C3
:1023D000050EDB50D880145406E2060EDB5003E1F4
:1023E000040EDB5034DA95D90AE2050EDBCFE7FFA5
:1023F000150EDB50E75E050EE7CFDBFF02D0050EC2
:10240000DB6A040EDBCF14F0160E45D9D8801454C5
:1024100014E2160EDBCFE6FF150EDBCFE6FF040E4F
:10242000DBCFE6FF050EDB50E552E75CE552D880D6
:10243000E754E552D880E7545FD9030EDB50010B17
:102440000BE1080EDB5008E0B2D801E08DD0080E99
:10245000DB50BED8080EDB6A170EDB5007E088D9C8
:10246000170EF1D903E1151C01E17ED0160EDB50E9
:1024700016E07ED9300EE66E9FD802E1151C74E09E
:1024800077D9DFCFE6FFACEC15F0E552E552E55227
:10249000F4CF15F00001F31C02E1151C65E0050EF8
:1024A000DBCF14F0160EDB50D880145409E2050E71
:1024B000DBCFE7FF160EDB50E75E050EE7CFDBFF55
:1024C000300EE66E050ECBD94FE1390EDB2ADBCF9D
:1024D000E9FF3A0E01E3DB2ADBCFEAFF090EEFCF7B
:1024E000DBFFDB500EE044D9090EADD902E1151C2B
:1024F0003BE0390EDB2ADBCFE9FF3A0EEDE3DB2AC6
:10250000EBD755D831E1160EDBCFE6FF080EC3D866
:10251000E552E7245DD82ED0070EDB50030A1CE0FD
:10252000010A14E0030A07E07BD9DBCFEEFF020EBD
:10253000DBCFEDFF1FD0F5D8196A17AE02D01868AF
:1025400019682CD8BCD819C0EEFF14D0EAD817BE31
:10255000186824D8B4D80ED063D9DBCFEFFF0AD0E7
:102560007BD905E1151C03E1F368F46810D0FCD8B1
:1025700001E3DB2A79D959EF0EF0010EDBCF14F01D
:10258000020EDBCF15F014C0F3FF15C0F4FF3B0EB5
:10259000E15C02E2E16AE552E16ECBD029D9020E9C
:1025A000BFEF13F061D90800F550DF6E1200200E66
:1025B000E66E080E2FEF14F0ACEC15F0E552E55284
:1025C000E552F3CF14F0F4CF15F00001F31C120024
:1025D000146E156AD950010F4DD91450EE261550BE
:1025E000ED221200185E000E195AF70E18C0DBFF1C
:1025F000F80E19C0DBFF18C0E9FF19C0EAFF12008E
:10260000DBCFF4FFF350F45C1200DB50E76E040EF6
:10261000E7CFDBFF12000A0EDBCF14F00B0EDBCF8F
:1026200015F00C0EDBCF16F00D0EDBCF17F01450AB
:102630001510161017101200130EEECFDBFF140E3C
:10264000EDCFDBFF130EDBCF14F0140EDBCF15F054
:102650000001800E15141200F70EDBCF18F0F80EF3
:10266000DBCF19F01200050EDB50E66ED950130FC8
:1026700001D9E552E750EE6EED6A12000A0EDBCF8B
:1026800006F00B0EDBCF07F00C0EDBCF08F00D0EC3
:10269000DBCF09F01200DBCFE6FF150EDBCFE6FF44
:1026A000050EDB50E552E724E552E7241200DB502B
:1026B000CED8010EF36E060EF3CFDBFF1200EE5004
:1026C000EFCFEAFFE96E16C0EEFF17C0EEFF18C0AD
:1026D000EEFF1200D9CFE6FFDACFE6FFE1CFD9FF58
:1026E000E2CFDAFF1200DFCFE6FFE66A93EC16F0E6
:1026F000E552E552F3501200E76E080EE7CFDBFF1C
:102700001200EECF14F0EECF15F0EFCF16F0176AEF
:102710001200050EDBCF14F0150EDB50D8801454D8
:102720001200010EDBCF16F0020EDBCF17F0186A95
:102730001200E552E5CFDAFFE7CFD9FF12000A0E0B
:1027400014C0DBFF0B0E15C0DBFF1200D9500A0FBF
:102750003AEF14F0F36E070EF3CFDBFF1200EECF6B
:1027600014F0EFCF15F01200010EDB2A020E12005A
:10277000FC0EDBCFE6FFFD0EDBCFE6FF1200145EA2
:10278000000E155AF70E14C0DBFFF80E15C0DBFF64
:1027900014C0E9FF15C0EAFF1200DA20EA6EEF2A42
:1027A000EECFF6FF000EEF22EECFF7FFEF22EECFD7
:1027B000F8FF1200040EDBCFE6FF130EDB50E552EC
:1027C000E75C9ADFDB5004DF060EDB501200090ED7
:1027D000DB500A0DF350DF24D00FE76E090EE7CF70
:1027E000DBFFD2EF12F0DB50F36E050E00EF13F0BB
:1027F000F70EDBCF14F0F80EDBCF15F01200DFCFB1
:10280000E6FFDCEF12F028DF030EECDE81EF13F0C1
:102810002EEC0EF0E552E552E552E55200091200A9
:10282000BDDEEE50EFCFEAFFE96E010E1200130E8F
:10283000DB50F36E040E00EF13F0040EDB50F36E6A
:10284000090E00EF13F0DBCFE6FFDCEF12F0E76ECE
:10285000050EE7CFDBFF12008BDFFFEF13F0DBCFBE
:10286000E6FF86DF08EF14F0D950F90FE96EFF0E8E
:0E287000CDEF13F0E96E000EDA20EA6E1200D2
:02287E00FF0E4B
:10288000E3CFEAFFE552FF0EE3CFE9FFE552E66A48
:10289000E66AD9CFE6FFDACFE6FFFC0EE124D96E77
:1028A000FF0EE220DA6EE66AE66AE66A200EEF5C68
:1028B00006E0090EEF5C03E0EF6603D03FD0EE5078
:1028C000F5D72D0EEF5C03E1FF0EE32A03D02B0EAC
:1028D000EF5C01E1EE502F0EEF6424D03A0EEF6072
:1028E00021D0D890F90EE336FA0EE336FD0EDECF96
:1028F000E3FFFE0EDDCFE3FFD890F90EE336FA0ECC
:10290000E336D890F90EE336FA0EE336FD0EE350C7
:10291000DE26FE0EE350DD22300EEE5CDE26000EDB
:10292000DD22D9D7FF0EE3CFE8FFE85207E0F90E2A
:10293000E31EE32AFA0ED8B4E306E31EE552E5529D
:10294000E552FF0EE3CFDAFFE552FF0EE3CFD9FFEA
:10295000E552E1CFE9FFE2CFEAFFED52ED52EECFD3
:08296000F3FFEFCFF4FF1200BA
:08296800D9CFE6FFDACFE6FF4C
:10297000E1CFD9FFE2CFDAFFE652E652E652E65265
:10298000D950F90F146EFF0EDA20156E020E14C026
:10299000DBFF030E15C0DBFF020EDBCFE6FF030EED
:1029A000DBCFE6FFF90EDBCFE6FFFA0EDBCFE6FF6B
:1029B000FB0EDBCFE6FFD950FC0FE66EFF0EDA20F0
:1029C000E66E44EC0EF0146E070EE15C02E2E16A82
:1029D000E552E16E1450F3CFDEFFF4CFDDFFFC0EC5
:1029E000DBCFE9FFFD0EDBCFEAFFEF6ADECF14F0AD
:1029F000DDCF15F014C0F3FF15C0F4FF040EE15C49
:102A000002E2E16AE552E16EE552E5CFDAFFE7CF97
:042A1000D9FF1200D8
:0C2A1400006A0EAE13EF15F00D6C0E1EE4
:102A2000E86A0E22001E09AE1BEF15F0086C091EA5
:102A3000E86A0922001E7DEC16F009BE2BEF15F0A6
:102A400000AE000C086C091EE86A0922046C051E21
:102A5000E86A0522000C00BE22EF15F00188FF0C89
:102A600009C013F008C012F008500D02F4CF07F0AF
:102A7000F3CF06F009500E02F4CF09F0F3CF08F0BF
:102A80000D02F3500726F4500822E86A092212507A
:102A90000E02F3500726F4500822E86A09220EAE0F
:102AA00056EF15F01250085E1350095A13AE000C81
:0A2AB0000D50085E0E50095A000C8C
:062ABA002A0EF66E080E64
:102AC000F76E000EF86E02010900F550056F09005F
:102AD000F550066F03E1056701D03DD00900F550C0
:102AE000006F0900F550016F0900F550026F0900F1
:102AF0000900F550E96E0900F550EA6E0900090079
:102B00000900F550036F0900F550046F0900090032
:102B1000F6CF07F2F7CF08F2F8CF09F200C2F6FFBE
:102B200001C2F7FF02C2F8FF0201035302E104539E
:102B300007E00900F550EE6E0307F8E20407F9D745
:102B400007C2F6FF08C2F7FF09C2F8FF0201050736
:082B5000000E065BBFD7120066
:082B5800D9CFE6FFDACFE6FF5A
:102B6000E1CFD9FFE2CFDAFFFB0EDBCF14F0FC0E92
:102B7000DBCF15F00001800E15141AE1FB0EDBCF40
:102B8000E9FFFC0EDBCFEAFFEECFF3FFEDCFF4FF62
:102B9000EE2A000EEF22F3CFE9FFF4CFEAFFFD0E9D
:102BA000DBCFEFFFEF50156AF36E15C0F4FF10D0C6
:102BB000FB0EDB50FE0806E1FD0EDBCFE6FFD3EC9B
:102BC00016F005D0FD0EDBCFE6FFF6EC16F0E55271
:0C2BD000E552E5CFDAFFE7CFD9FF120095
:042BDC0006500B0292
:102BE000F3CF02F0F4CF03F00C02F3500326000EF3
:102BF000F420046E06500D02F3500426000EF4205B
:102C0000056E06500E02F350052607500B02F350D6
:102C10000326F4500422000E052207500C02F35044
:102C20000426F450052207500D02F35005260850E3
:102C30000B02F3500426F450052208500C02F35006
:0C2C4000052609500B02F3500526120077
:042C4C00FE0EE3CFC6
:102C5000E9FFFF0EE3CFEAFFF36AF46AEE5203E006
:102C6000F34AF42AFBD71200FF0EE3CFF8FFE55238
:102C7000FF0EE3CFF7FFE552FF0EE3CFF6FFE5527D
:102C8000E66AE66AE66A0900F55209E0FD0EE32A03
:102C900005E1FE0EE32A02E1FF0EE32AF4D7FD0E62
:102CA000E3CF07F0FE0EE3CF08F0FF0EE3CF09F00D
:022CB000120010
:0E2CB200056A046A036A026A200EE76ED89073
:102CC0000636073608360936023603360436053628
:102CD0000B50025C0C5003580D5004580E50055810
:102CE00009E30B50025E0C50035A0D50045A0E506B
:0A2CF000055A062AE72EE4D7120069
:062CFA00056A046A100ED9
:102D0000E76ED89008360936043605360D50045C57
:102D10000E50055805E30D50045E0E50055A082A62
:062D2000E72EF0D71200BF
:0A2D2600F36AF46AFF0EE124E96E7F
:102D3000FF0EE220EA6EED6607D02F0EEF6404D09E
:0A2D40003A0EEF6001D0F32A1200F2
:062D4A00FF0EE3501B6EBA
:102D5000480E01D04C0EE76EE72EFED7E76AE72E4D
:0A2D6000FED71B2EF7D7000012006B
:062D6A00000EF36E00EE06
:102D700000F0080E01D81200EA6002D0EE6AFCD71B
:0A2D8000F350E9601200EE6AFCD780
:062D8A0012EE40F022EE03
:102D900040F0F86A019C5DEC15F0F7EC16F066EC7B
:062DA0000DF0FBD712004C
:0A2DA600FF0EE350ACBA04D0AF6A90
:102DB000AB8EAC8A949CACA2FED7AD6EF36EF46A77
:022DC0001200FF
:0E2DC200FF0EE350E84E1200000000D000D0DB
:082DD00000D0E82EFAD7120032
:082DD800303132333435363757
:092DE00038396162636465660024
:032DE9002564005E
:022DEC001200D3
:022DEE001200D1
:102DF000EEEDEBE7DEDDDBD7BEBDBBB77E7D7B77DF
:102E00003031323334353637383941424344454620
:102E10000000303000FC121212FCFE9292926C7C88
:102E200082828244FE8282827CFE92929282FE1292
:102E30001212027C92929274FE101010FE0082FE1A
:102E40008200708080807EFE10284482FE80808018
:102E500080FE041804FEFE081020FE7C8282827C24
:102E6000FE1212120CFC82A242BCFE1232528C4C98
:102E7000929292640202FE02027E8080807E3E4038
:102E800080403EFE403040FEC6281028C60608F0AE
:102E90000806C2A2928A867C8282827C0084FE809E
:102EA0000084C2A2928C448292926C1E101010FE7A
:102EB0005E929292627C92929264824222120E6C94
:092EC0009292926C4C9292927C69
:00000001FF
